:1000000018308A000E2E0000FF00030E8301A100AD
:100010000A08A0008A010408A2007708A300780853
:10002000A4007908A5007A08A6007B08A70083131E
:1000300083128C308400801E1F288C1A32282208DC
:1000400084002308F7002408F8002508F900260892
:10005000FA002708FB0020088A00210E8300FF0E0B
:100060007F0E09008A110A12FF280A108A100A114D
:1000700082074F344E3434344934593420345234A6
:1000800042344F3458342D343334303461344434B2
:10009000573400340A108A100A1182074E344F3444
:1000A0002034573441345234523441344E34543471
:1000B00049344534533420344F34523400340A1018
:1000C0008A100A118207203443344F344D344D34A2
:1000D000453452344334493441344C34203455345B
:1000E00053344534203400340A108A100A11820730
:1000F00020344F34443444342034203400340A1043
:100100008A100A11820720344534563445344E345F
:10011000203400340A108A100A11820749344E3400
:10012000563441344C3400340A108A100A118207C4
:100130002034203400340A108A100A118207203437
:10014000533441345434533400340A108A100A11A1
:100150008207483444344F345034203400340A1079
:100160008A100A11820753344534523449344134D9
:100170004C3420344F344B3400340A108A100A11A6
:1001800082074E344F3454342034413420344734C1
:100190005034533400340A108A100A11820747344D
:1001A00050345334203446344F3455344E34443470
:1001B00000340A108A100A1182074734503452342E
:1001C0004D34433420345034463400340A108A10FD
:1001D0000A118207473450344734473441342034BD
:1001E0005034463400340A108A100A1182074E3403
:1001F0004F3420344734503453343F340034831662
:1002000086108312861428302C0784008C1E062941
:100210001A0880002C088316E900013083122C078D
:100220000339AC002D082C02031D1A298316690816
:100230008312AC0083168610831286108C128A11EA
:100240000A121F286430840000080319362901307F
:10025000F800F701F70B2A29F80B29296630F70077
:10026000F70B302900000000800B272900340E30E6
:10027000F700F70B392974081039003A031D422999
:100280000812432908168316081274082039003A08
:10029000031D4E2983128812502983168312881653
:1002A0008316881274084039003A031D5B298312B3
:1002B00008135D2983168312081783160813740820
:1002C0008039003A031D6829831288136A2983162E
:1002D0008312881783168813881183128815831652
:1002E00088118312881174080139003A031D7A2994
:1002F00008127B2908168316081274080239003A7E
:10030000031D862983128812882983168312881672
:100310008316881274080439003A031D9329831246
:100320000813952983168312081783160813740877
:100330000839003A031DA02983128813A2298316C5
:1003400083128817831688138811831288158316E1
:100350008811831288110034831688108312881044
:100360000830F40037210130F40037210230E40076
:1003700022210230F40037210230E400222106302D
:10038000F40037210C30F40037210230E400222140
:10039000003483168810831288147308F400372100
:1003A0000034831688108312881080306B07EC00AD
:1003B000F4003721003483161F149F141F159F115A
:1003C00083121F108316091283129412DD125D0826
:1003D0008316870083125D165D08831687008312DB
:1003E000DD115D08831687000030831294008316A8
:1003F00094000108C7390838810083129001003049
:10040000F800920000308316920083125D155D089B
:1004100083168700831297019701DD145D08831608
:10042000870083129D019D01073083169C000508FB
:100430000330F700F70B1A2A1C0883120D138316DA
:100440009D018C16C03083128B0483160610831214
:1004500006148316861083128610831606118312E3
:1004600006118316861183128611831606128312D3
:10047000061283168612831286120330E300831657
:1004800088108312881083168811831288118316AE
:100490000811831208110F30E4002221630801398A
:1004A000003A031D552A0812562A08168316081208
:1004B000831263080239003A031D602A8812612AF8
:1004C000881683168812831263080439003A031DC4
:1004D0006B2A08136C2A0817831608138312630803
:1004E0000839003A031D762A8813772A881783165D
:1004F0008813881183128815831688118312881136
:100500000530E400222163080139003A031D8A2ADC
:1005100008128B2A08168316081283126308023900
:10052000003A031D952A8812962A88168316881287
:10053000831263080439003A031DA02A0813A12A74
:10054000081783160813831263080839003A031D3D
:10055000AB2A8813AC2A8817831688138811831254
:10056000881583168811831288110530E400222132
:1005700063080139003A031DBF2A0812C02A081671
:1005800083160812831263080239003A031DCA2A2F
:100590008812CB2A881683168812831263080439BE
:1005A000003A031DD52A0813D62A08178316081304
:1005B000831263080839003A031DE02A8813E12AF0
:1005C000881783168813881183128815831688115B
:1005D000831288110530E4002221081283160812C4
:1005E0008312881683168812831208138316081341
:1005F0008312881383168813881183128815831633
:100600008811831288112830F4003721AC21E301CE
:100610006308352000380319112BE30AF300C921C0
:10062000082B0330E300FA30E4002221E30B132B04
:100630004030EB00D121E30163084A200038031960
:10064000252BE30AF300C9211C2B83160610831205
:1006500006100230E300FA30E4002221E30B2B2BDA
:1006600083160610831206104030EB00D121E301FF
:1006700063085F2000380319412BE30AF300C92106
:10068000382B0230E300FA30E4002221E30B432B45
:1006900083160610831206148A150A16312E2D08A9
:1006A0002C0203194F2B28302D0784000008EB0083
:1006B00001302D070339AD006B08F80000346910D4
:1006C000E801E8016808E80A003A0319742B63306E
:1006D0006807EA004F236A088400780880006808E9
:1006E000033C031C0030622B6918972B4F237808BA
:1006F000E7006308473C031D8D2B6408503C031D35
:100700008D2B6508523C031D8D2B66084D3C031D47
:100710008D2B6708433C03196914E80A6408E30059
:100720006508E4006608E5006708E600742B003001
:1007300069180130F80000344F237808E400640899
:100740002C3C0319A72B4F237808E4009F2B00347F
:100750004F234F237808AE004F237808AF004F2374
:100760007808B0004F237808B1004F237808B20012
:100770004F237808B3000330B30730303302093C0D
:100780000318C52B0A30B302B20A30303202053CDE
:100790000318CF2B3030B2003108B10AB10030302D
:1007A0003102093C0318D72B0A30B102B00A3030AD
:1007B0003002053C0318DF2B3030B000AF0A9C2319
:1007C0004F237808413C031DE72B5C14E82B5C1099
:1007D0009C234F237808B4004F237808B5004F239B
:1007E0007808B6004F237808B7004F234F237808C6
:1007F000B8009C239C234F237808B9004F23780826
:10080000BA004F237808BB004F237808BC004F2361
:100810007808BD009C234F237808BE009C239C23AE
:100820009C234F237808BF004F237808C0004F2334
:100830007808C1004F237808C2008A150A16E12EF5
:10084000F701F801700803107118F707F70CF80C9E
:10085000F118F707F70CF80C7119F707F70CF80CFB
:10086000F119F707F70CF80C711AF707F70CF80CE9
:10087000F11AF707F70CF80C711BF707F70CF80CD7
:10088000F11BF707F70CF80C00348E30F7008316D5
:100890005308F8005208F900FA01F808031D5A2C11
:1008A0007908F800F9010830F702F808031D5A2CFE
:1008B000F701622C0310F81B612CF90DF80DF703FA
:1008C0005A2CF8130000831200348030831C6B2CE8
:1008D0008316D80683128316DD01DE015408DC007E
:1008E0005808DC0653080319562DDB00F70057089B
:1008F00003195F2DDB020319FC2C031CBB2C5808C9
:10090000E100E1175908E0005A08DF00DE0103109A
:10091000E10CE00CDF0CDE0CDB0B862CDC1F932CD7
:100920005D14732D5D105B105D16D6308400882D2C
:100930005D12DC1BA52C5B1CB02CE10CE00CDF0C69
:10094000DE0CF70A03196E2DB02CE11BB32C03103B
:10095000DE0DDF0DE00DE10DF70303196E2DA52C63
:100960005D171B2D5D135408DC00D41FB92CE11753
:10097000672DE113672D5708DB00F7005308DB02F2
:100980005408E100E1175508E0005608DF00DE01D9
:100990000310E10CE00CDF0CDE0CDB0BC72CDC1FC2
:1009A000D42CDD14732DDD105B10DD16DA308400DD
:1009B000882DDD12DC1BE62C5B1CF12CE10CE00C1D
:1009C000DF0CDE0CF70A03196E2DF12CE11BF42C61
:1009D0000310DE0DDF0DE00DE10DF70303196E2DA1
:1009E000E62CDD171B2DDD135808DC00D81FFA2C70
:1009F000E117672DE113672D5808E100E117590849
:100A0000E0005A08DF00DC1F092DE1135D15732D8E
:100A10005D11DE015B10D6308400882DDC1B312D8A
:100A20005408DC005B1C1B2DE10CE00CDF0CDE0C21
:100A3000F70A03196E2DDE1F2C2DDF0A031D2C2D46
:100A4000E00A031D2C2DE10A031D2C2DE10CE00C06
:100A5000DF0CF70A03196E2D5D1BB22CDD1BF32C86
:100A6000502D8030E106E11F392D732D5808DC0030
:100A7000462D5408DC00E108031D462DE008031D47
:100A8000462DDF08031D462DF701672DE11B502D74
:100A90000310DE0DDF0DE00DE10DF70B462D6E2D81
:100AA000DC1F542DE117672DE113672D5708F70060
:100AB0005808E1005908E0005A08DF00672D530884
:100AC000F7005408E1005508E0005608DF0061080F
:100AD000F8006008F9005F08FA00A62DF701F80198
:100AE000F901FA01A62DDE01DF09E009E109DE09BD
:100AF000DE0A031D812DDF0A031D812DE00A031983
:100B0000E10A5D18922CDD18D32C5D19082D362DC5
:100B10000008DF07031C922DE00A031D922DE10A55
:100B200003195B1484030008E007031C9A2DE10AF3
:100B300003195B1484030008801F803AE10703183F
:100B40005B145D1A982CDD1AD92C0E2D000083122F
:100B5000003483164E0803196F2EDA005208031969
:100B60006F2EDA02031CB92D7F30DA0703186F2EBF
:100B7000BF2D8130DA02031C6F2E03196F2E5A0825
:100B8000F700F801F901FA01D9014F08D800D81788
:100B90005008D7005108D6001930DA005508D6029F
:100BA0000318E22D0130D7020318E22DD8020318F2
:100BB000E22DD9020318E22DD90AD80AD70A55081E
:100BC000D607142E5408D7020318FD2D0130D80281
:100BD0000318FD2DD9020318FD2DD90AD80A54088F
:100BE000D7075508D607031C142ED70A031D142E49
:100BF000D80A031D142ED90A142E53088038D8029F
:100C00000318132E0130D9020318132ED90A5308E2
:100C10008038D8075408D707031CF12DD80A031DC4
:100C2000F12DD90AF12D7A14DA0B172E222E03108A
:100C3000D60DD70DD80DD90D0310FA0DF90DF80DFD
:100C4000DB0DCE2D5B1C2A2E0310F80CF90CFA0CD0
:100C5000DB0C2D2EF70303196F2EDB1B562E031012
:100C6000D60DD70DD80DD90D5508D6020318422E32
:100C70000130D7020318422ED8020318422ED9029F
:100C8000031C652E5408D70203184D2E0130D802DC
:100C900003184D2ED902031C652E53088038D80244
:100CA0000318562E0130D902031C652EFA0A031DC3
:100CB000652EF90A031D652EF80A031D652EF70A35
:100CC00003196F2EF80CF90CFA0C4F08DA005308D0
:100CD000DA06DA1F6D2EF817732EF813732EF7014C
:100CE000F801F901FA01000083120034831652085A
:100CF0000319E72EDA0056080319E72EDA0703185E
:100D0000882E7F30DA02031CE72E0319E72E8C2E83
:100D10008130DA070318E72E5A08F700F801F901C5
:100D2000FA015308DE00DE175408DD005508DC0028
:100D30001830DA00DB015C1CB52E5908FA07031CD9
:100D4000A72EF90A031DA72EF80A0319DB17580866
:100D5000F907031CAE2EF80A0319DB175708D40055
:100D6000D4175408F8070318DB17DB0DF80CF90C3F
:100D7000FA0CDE0CDD0CDC0C0310DA0B9A2E0130C1
:100D8000F7070318E72EF81BCC2EDE0DFA0DF90D30
:100D9000F80DF7030319E72EDE1FDD2EFA0A031DF7
:100DA000DD2EF90A031DDD2EF80A031DDD2EF80CD9
:100DB000F90CFA0CF70A0319E72E5308DB00570861
:100DC000DB06DB1FE52EF817EB2EF813EB2EF701F1
:100DD000F801F901FA0100008312003483164F086C
:100DE000D6005308D606D61FFA2E03110310CF1BC8
:100DF00003142D2F4F08D6005208D7004E08D702F3
:100E00000319082FD61F2D2F0308013A83002D2F19
:100E10005308D7004F08D7020319142FD61F2D2FC0
:100E20000308013A83002D2F5408D7005008D70239
:100E30000319202FD61F2D2F0308013A83002D2FD1
:100E40005508D7005108D70203192C2FD61F2D2F74
:100E50000308013A83002D2F0310831200348E30D3
:100E6000F70083164E08F7024F08F9005008F80003
:100E7000F917F7080319472F0310F908031D432F2B
:100E8000F8080319472FF90CF80CF70B3C2FCF1F6C
:100E90004E2FF809F909F80A0319F90A000083121C
:100EA0000034831483162308D6002208D5002108B5
:100EB000D4002008D300DB30DA000F30D9004930ED
:100EC000D8007F30D7008312652477088316A400EA
:100ED0007808A5007908A6007A08A700AB002608C4
:100EE000AA002508A9002408A8008A158312552104
:100EF0008A1100347208F80171020318822F7108F8
:100F0000F7008E2FF7010830F300F10DF70D72088E
:100F100077020318F700F80DF30B852F003410301B
:100F2000F700FA01EF01EC0CEB0C031C9D2F6D0890
:100F3000FA070318EF0A6E08EF07EF0CFA0CF90C2A
:100F4000F80CF70B932F8A110A16FD28F801F90106
:100F5000F701FA016C08031DB02F6B080319CA2FA3
:100F60001030ED000310E90DEA0DF70DFA0D6C08D5
:100F70007A02031DBD2F6B087702031CC62F6B0876
:100F8000F702031CFA036C08FA020314F80DF90DBA
:0C0F9000ED0BB22F00008A110A16E429B4
:1010000030304102E800F0000A30F1008A1120245B
:101010008A157808E900303042026907E300303071
:101020003F02E800F0000A30F1008A1120248A15FE
:101030007808E900303040026907E4006308013AAB
:1010400003194428033A03194828013A03194D2883
:10105000073A03195228013A03195728033A03198A
:101060005C28013A031961280F3A03196628013AEE
:1010700003196B28033A03197028013A03197828D9
:10108000073A031980288828E6016408E5008B28C0
:101090001F306407E500E6018B283B306407E5005C
:1010A000E6018B285A306407E500E6018B2878308A
:1010B0006407E500E6018B2897306407E500E60148
:1010C0008B28B5306407E500E6018B28D43064072F
:1010D000E500E6018B28F3306407E500E6018B2884
:1010E00011306407E5000130E6000318E60A8B289A
:1010F00030306407E5000130E6000318E60A8B286B
:101100004E306407E5000130E6000318E60A8B283C
:10111000E6010130E50030302E02E800F0000A3030
:10112000F1008A1120248A157808E90030302F0256
:1011300069078316D301D2008A11831245248A15C8
:101140007A08D1007908D0007808CF007708CE005F
:1011500001306502E7006608E8000030031C01303A
:10116000E802831451088316D600831250088316B0
:10117000D50083124F088316D40083124E088316BD
:10118000D300DA01D9014030D8008230D7008A116B
:10119000831265248A157708E9007808EA0079083F
:1011A000EB007A08EC008316D10083126B088316DB
:1011B000D00083126A088316CF0083126908831651
:1011C000CE00D501D4014030D3008330D2008A1143
:1011D0008312A9258A157708ED007808EE007908B2
:1011E000EF007A08F00068088316D30083126708BE
:1011F0008316D2008A11831245248A1583107A0837
:101200008316D6007908D5007808D4007708D30073
:101210007008DA0083126F088316D90083126E08F3
:101220008316D80083126D088316D7008A118312A3
:1012300065248A157708F1007808F2007908F30030
:101240007A08F4008316D1007308D0007208CF002A
:101250007108CE00D5018030D4003630D3008730FD
:10126000D2008A118312A9258A15DB308316D50096
:101270000F30D4004930D3008130D2007A08D90031
:101280007908D8007808D7007708D6008A11831229
:1012900076268A157A08D1007908D0007808CF0020
:1012A0007708CE008A150A16FA2E7F308316B4000E
:1012B000B501B601B7017E30BE008030BF00C0016D
:1012C000C1017A30C2002A30C300AA30C400A33062
:1012D000C5007530C600B630C7000930C8009C3064
:1012E000C9006F30CA004F30CB00B430CC000B3097
:1012F000CD002B08D1002A08D0002908CF002808EB
:10130000CE00D501D401D301D2018A118312EE2679
:101310008A15031C8F2980308316A9068312831631
:101320002B08D1002A08D0002908CF002808CE00B9
:10133000DB30D5000F30D4004930D3007F30D200ED
:101340008A118312A9258A157A088316D100790893
:10135000D0007808CF007708CE008A1183122F279B
:101360008A1578088316B8002B08D1002A08D00007
:101370002908CF002808CE00DB30D5000F30D4007C
:101380004930D3007F30D2008A118312A9258A15F3
:1013900077088316CE007808CF007908D0007A0845
:1013A000D100D3013808D2008A11831245248A154E
:1013B000831483165108D6005008D5004F08D40076
:1013C0004E08D3007A08DA007908D9007808D800E6
:1013D0007708D7008A11831265248A157A08831644
:1013E000BD007908BC007808BB007708BA0003305C
:1013F000B805B8080319002A3808023C031D1E2A44
:101400003D08D5003C08D4003B08D3003A08D20080
:10141000DB30D9000F30D8004930D7007F30D600FC
:101420008A11831276268A157A088316B300790802
:10143000B2007808B1007708B0008F2A380B582A1C
:101440008314D601D501D4017F30D3003D08DA00E2
:101450003C08D9003B08D8003A08D7008A1183120B
:1014600065248A1577088316CE007808CF0079089E
:10147000D0007A08D100D5005008D4004F08D3001E
:101480004E08D200DB30D9000F30D8004930D700E9
:101490007F30D6008A11831276268A157A08831641
:1014A000B3007908B2007808B1007708B0008F2A3D
:1014B00083143D08D6003C08D5003B08D4003A0808
:1014C000D300DA01D901D8017F30D7008A11831205
:1014D00065248A1577088316CE007808CF0079082E
:1014E000D0007A08D100D5005008D4004F08D300AE
:1014F0004E08D200DB30D9000F30D8004930D70079
:101500007F30D6008A11831276268A157A088316D0
:10151000B3007908B2007808B1007708B000AF01D5
:10152000AE01AD017F30AC003308D5003208D400E5
:101530003108D3003008D2003308D9003208D8006F
:101540003108D7003008D6008A11831276268A1512
:101550007A088316B3007908B2007808B1007708DA
:10156000B000B9013908033C031C1E2B3708D50015
:101570003608D4003508D3003408D2003308D90027
:101580003208D8003108D7003008D6008A118312FB
:1015900076268A157A088316B7007908B600780887
:1015A000B5007708B400390DF700F70DFC30F705EA
:1015B0007708BE3E84000008CE00840A0008CF00F1
:1015C000840A0008D000840A0008D100D500500821
:1015D000D4004F08D3004E08D2003708D90036088F
:1015E000D8003508D7003408D6008A118312762631
:1015F0008A1504088316D20083102F08D6002E08FF
:10160000D5002D08D4002C08D3007A08DA00790818
:10161000D9007808D8007708D7008A11831265248A
:101620008A158316520884007A08AF007908AE0044
:101630007808AD007708AC00B90AB22A3808023C35
:101640000319242B380B262B8030AD062C08F7000D
:101650002D08F8002E08F9002F08FA008312003434
:1016600051088316AB00831250088316AA00831218
:101670004F088316A90083124E088316A800831210
:1016800055217A08E6007908E5007808E400770833
:10169000E30051088316A300831250088316A200AA
:1016A00083124F088316A10083124E088316A000F0
:1016B0008A11831251278A157A08EA007908E9000D
:1016C0007808E8007708E70051088316D5008312F0
:1016D00050088316D40083124F088316D300831258
:1016E0004E088316D200D901D801D7018030D60028
:1016F0008A11831276268A157708F3007808F40099
:101700007908F5007A08F6008316AB007508AA0080
:101710007408A9007308A800831255217A08EE0006
:101720007908ED007808EC007708EB005108831683
:10173000D500831250088316D40083124F088316F5
:10174000D30083124E088316D200D901D801D701E5
:101750008030D6008A11831276268A157708F30026
:101760007808F4007908F5007A08F6008316A300DB
:101770007508A2007408A1007308A0008A118312E2
:1017800051278A157A08F2007908F1007808F000EC
:101790007708EF005230D5004930D4001D30D30017
:1017A0007130D200AE308316D500D730D4007430FB
:1017B000D3007530D200831266088316D9008312D5
:1017C00065088316D800831264088316D700831235
:1017D00063088316D6008A11831276268A15831031
:1017E00055088316D600831254088316D500831239
:1017F00053088316D400831252088316D3007A0844
:10180000DA007908D9007808D8007708D7008A115B
:10181000831265248A157A08D5007908D4007808DF
:10182000D3007708D2002C308316D5006330D40063
:101830000330D3007A30D20083126A088316D900AD
:10184000831269088316D800831268088316D700AC
:10185000831267088316D6008A11831276268A15AA
:10186000831455088316D600831254088316D500B6
:10187000831253088316D400831252088316D300B0
:101880007A08DA007908D9007808D8007708D700F4
:101890008A11831265248A157A08D5007908D40044
:1018A0007808D3007708D200C1308316D500733092
:1018B000D4006F30D3007830D20083126E088316C4
:1018C000D90083126D088316D80083126C08831622
:1018D000D70083126B088316D6008A1183127626EE
:1018E0008A15831455088316D6008312540883166C
:1018F000D500831253088316D4008312520883162E
:10190000D3007A08DA007908D9007808D800770877
:10191000D7008A11831265248A157A08D5007908C0
:10192000D4007808D3007708D20048308316D50059
:101930005130D4002730D3007A30D2007208D90059
:101940007108D8007008D70083126F088316D6007C
:101950008A11831276268A15831455088316D600B9
:10196000831254088316D500831253088316D400BB
:10197000831252088316D3007A08DA007908D90056
:101980007808D8007708D7008A11831265248A1551
:101990007A08D5007908D4007808D3007708D200F7
:1019A00055088316D500831254088316D400831279
:1019B00053088316D300831252088316D2001430C2
:1019C000D9002E30D8006530D7008630D6008A1175
:1019D000831276268A157A08D5007908D40078080B
:1019E000D3007708D2008A150A16FD2E51088316F7
:1019F000AB00831250088316AA0083124F08831687
:101A0000A90083124E088316A800831255217A0874
:101A1000E6007908E5007808E4007708E30051085B
:101A20008316A300831250088316A20083124F0866
:101A30008316A10083124E088316A0008A11831218
:101A400051278A157A08EA007908E9007808E80041
:101A50007708E70051088316D500831250088316D3
:101A6000D40083124F088316D30083124E088316C6
:101A7000D200D901D801D7018030D6008A11831253
:101A800076268A157708F3007808F4007908F500BF
:101A90007A08F6008316AB007908AA007808A90036
:101AA0007708A800831255217A08EE007908ED0026
:101AB0007808EC007708EB0051088316D5008312F4
:101AC00050088316D40083124F088316D300831264
:101AD0004E088316D200D901D801D7018030D60034
:101AE0008A11831276268A157708F3007808F400A5
:101AF0007908F5007A08F6008316A3007908A20099
:101B00007808A1007708A0008A11831251278A154E
:101B10007A08F2007908F1007808F0007708EF0001
:101B20006430D900B030D8006230D7007730D600AA
:101B300044308316D500C130D4004C30D3007D3002
:101B4000D200831266088316D900831265088316B3
:101B5000D800831264088316D700831263088316A3
:101B6000D6008A11831276268A15831459088316A3
:101B7000D600831258088316D5008312570883169F
:101B8000D400831256088316D3007A08DA00790845
:101B9000D9007808D8007708D7008A118312652405
:101BA0008A157A08D9007908D8007808D70077080C
:101BB000D600E7308316D500E230D4000F30D300D2
:101BC0007B30D20083126A088316D9008312690819
:101BD0008316D800831268088316D700831267081B
:101BE0008316D6008A11831276268A158310590827
:101BF0008316D600831258088316D500831257081F
:101C00008316D400831256088316D3007A08DA00AC
:101C10007908D9007808D8007708D7008A1183128C
:101C200065248A157A08D9007908D8007808D70081
:101C30007708D60036308316D5007230D4005D3078
:101C4000D3007730D20083126E088316D900831236
:101C50006D088316D80083126C088316D700831290
:101C60006B088316D6008A11831276268A15831490
:101C700059088316D600831258088316D50083129C
:101C800057088316D400831256088316D3007A08A7
:101C9000DA007908D9007808D8007708D7008A11C7
:101CA000831265248A157A08D9007908D800780843
:101CB000D7007708D600BD308316D500C330D400D6
:101CC0006D30D3007430D2007208D9007108D8008A
:101CD0007008D70083126F088316D6008A1183120A
:101CE00076268A15831059088316D6008312580861
:101CF0008316D500831257088316D4008312560822
:101D00008316D3007A08DA007908D9007808D80059
:101D10007708D7008A11831265248A157A08D900BA
:101D20007908D8007808D7007708D6008316D5013F
:101D3000D4014030D3008030D20083125108831682
:101D4000D900831250088316D80083124F088316D7
:101D5000D70083124E088316D6008A118312762686
:101D60008A157708F3007808F4007908F5007A08F6
:101D7000F6008316AB007908AA007808A900770856
:101D8000A8008312552127308316D500C030D40017
:101D90003030D3007630D2007A08D9007908D800E4
:101DA0007808D7007708D6008A11831276268A151C
:101DB0000408F400831459088316D60083125808C7
:101DC0008316D500831257088316D4008312560851
:101DD0008316D3007A08DA007908D9007808D80089
:101DE0007708D7008A11831265248A157408840045
:101DF0007A08D9007908D8007808D7007708D60083
:101E00008316D501D4014030D3008030D200831234
:101E100051088316D900831250088316D800831204
:101E20004F088316D70083124E088316D6008A11F6
:101E3000831276268A157708F3007808F40079086B
:101E4000F5007A08F6008316A3007908A200780846
:101E5000A1007708A0008A11831251278A158F30BC
:101E60008316D500FC30D4004130D3007530D20049
:101E70007A08D9007908D8007808D7007708D60002
:101E80008A11831276268A150408F40083105908F3
:101E90008316D600831258088316D500831257087C
:101EA0008316D400831256088316D3007A08DA000A
:101EB0007908D9007808D8007708D7008A118312EA
:101EC00065248A15740884007A08D9007908D80036
:101ED0007808D7007708D6008A150A16002F51080F
:101EE0008316D100831250088316D00083124F0846
:101EF0008316CF0083124E088316CE00D501D4017D
:101F0000D3018130D2008A118312A9258A1577085E
:101F1000E3007808E4007908E5007A08E600831415
:101F200066088316D600831265088316D5008312CF
:101F300064088316D400831263088316D300DA0181
:101F4000D9013430D8008630D7008A118312652435
:101F50008A157708E7007808E8007908E9007A0828
:101F6000EA008316D500831269088316D400831211
:101F700068088316D300831267088316D200DB300B
:101F8000D9000F30D8004930D7008030D6008A11F0
:101F9000831276268A157708EB007808EC0079081A
:101FA000ED007A08EE008316D10083126D088316C7
:101FB000D00083126C088316CF0083126B0883163F
:101FC000CE00D501D4013430D3008630D2008A113E
:101FD0008312A9258A157A08D1007908D0007808DB
:0C1FE000CF007708CE008A150A16062FE5
:1020000030302E02EC00F0000A30F1000A122024D9
:102010000A167808ED0030302F026D07E700E8015E
:1020200030303002EC00F0000A30F1000A122024B7
:102030000A167808ED00303031026D07E9003030C3
:102040003902EC00F0006430F1000A1220240A1674
:102050007808ED0030303A02EF00F0000A30F1006D
:102060000A1220240A1678086D07F00030303B026F
:1020700070078316D301D2000A12831245240A1670
:102080007A08E6007908E5007808E4007708E300BC
:1020900030303C02EC00F0000A30F1000A1220243B
:1020A0000A163D087807D03EF000F1003C30F200FF
:1020B0000A127A270A1678088316D301D2000A1268
:1020C000831245240A16831066088316D6008312ED
:1020D00065088316D500831264088316D400831222
:1020E00063088316D3007A08DA007908D9007808E3
:1020F000D8007708D7000A12831265240A167A08D6
:10210000E6007908E5007808E4007708E3003E0877
:10211000573C031DAE288316D501D4018030D3006F
:102120007F30D200831266088316D90083126508B7
:102130008316D800831264088316D70083126308BD
:102140008316D6000A12831276260A167A08E6004B
:102150007908E5007808E4007708E3008316D501E4
:10216000D401D3018130D200831266088316D900CE
:10217000831265088316D800831264088316D7007B
:10218000831263088316D6000A12831276260A1673
:10219000831055088316D600831254088316D50081
:1021A000831253088316D400831252088316D30077
:1021B0007A08DA007908D9007808D8007708D700BB
:1021C0000A12831265240A167A08D1007908D00011
:1021D0007808CF007708CE005108E6005008E500E7
:1021E0004F08E4004E08E3006808EC006708EB00C5
:1021F000EE013C30ED000A128F2F0A167908FA0022
:1022000078088316D2007908D3000A128312452475
:102210000A16831066088316D60083126508831693
:10222000D500831264088316D400831263088316D2
:10223000D3007A08DA007908D9007808D80077083E
:10224000D7000A12831265240A167708EB00780873
:10225000EC007908ED007A08EE008316D3018312B2
:1022600069088316D2000A12831245240A168310C5
:102270006E088316D60083126D088316D50083126C
:102280006C088316D40083126B088316D3007A0877
:10229000DA007908D9007808D8007708D7000A1240
:1022A000831265240A167A08D1007908D0007808CC
:1022B000CF007708CE0051088316D1008312500852
:1022C0008316D00083124F088316CF0083124E0866
:1022D0008316CE00D501D4013430D3008830D2002B
:1022E0000A128312EE260A16031C7829DC147929B7
:1022F000DC108A150A16032F30303402E800F00093
:102300000A30F1000A1220240A167808E900303059
:10231000350269078316D301D2000A1283124524BD
:102320000A167A08E6007908E5007808E4007708DC
:10233000E30030303602E800F0000A30F1000A1203
:1023400020240A1637087807D03EEC00F1003C3014
:10235000F2000A127A270A1678088316D301D200EF
:102360000A12831245240A16831066088316D600C3
:10237000831265088316D500831264088316D4007F
:10238000831263088316D3007A08DA007908D9002B
:102390007808D8007708D7000A12831265240A1635
:1023A0007A08E6007908E5007808E4007708E30099
:1023B00030303802E800EA016808E9000230EC0039
:1023C0005830EB000A12A62F0A167908FA0078088E
:1023D0008316D2007908D3000A12831245240A1604
:1023E000831066088316D600831265088316D5000D
:1023F000831264088316D400831263088316D30003
:102400007A08DA007908D9007808D8007708D70068
:102410000A12831265240A167A08E6007908E50094
:102420007808E4007708E30066088316D500831275
:1024300065088316D400831264088316D3008312C0
:1024400063088316D200DB30D9000F30D800493042
:10245000D7008030D6000A12831276260A16770833
:10246000E7007808E8007908E9007A08EA008316AE
:10247000D100831269088316D0008312680883167E
:10248000CF00831267088316CE00D501D401343003
:10249000D3008630D2000A128312A9250A167A08C0
:1024A000E6007908E5007808E4007708E3006608AC
:1024B000D5006508D4006408D3006308D200510831
:1024C0008316AB00831250088316AA0083124F08AC
:1024D0008316A90083124E088316A8000A128A15D3
:1024E000831255210A168A117A08D1007908D00082
:1024F0007808CF007708CE0066088316AB008312F9
:1025000065088316AA00831264088316A900831243
:1025100063088316A8000A128A15831255210A1629
:102520008A117708E7007808E8007908E9007A0856
:10253000EA0059088316AB00831258088316AA00D4
:10254000831257088316A900831256088316A80021
:102550000A128A15831255210A168A116A088316EF
:10256000D500831269088316D40083126808831685
:10257000D300831267088316D2007A08D90079083D
:10258000D8007808D7007708D6000A12831276267A
:102590000A167708EB007808EC007908ED007A0855
:1025A000EE008316D50083126D088316D4008312C3
:1025B0006C088316D30083126B088316D200831233
:1025C00051088316D900831250088316D80083124D
:1025D0004F088316D70083124E088316D6000A12BE
:1025E000831276260A167A08D1007908D000780876
:1025F000CF007708CE0066088316A3008312650813
:102600008316A200831264088316A1008312630854
:102610008316A0000A12831251270A167708E700D2
:102620007808E8007908E9007A08EA005908831672
:10263000A300831258088316A2008312570883163A
:10264000A100831256088316A0000A128312512794
:102650000A166A088316D500831269088316D40007
:10266000831268088316D300831267088316D2008A
:102670007A08D9007908D8007808D7007708D600FA
:102680000A12831276260A160408EB0083105108FA
:102690008316D600831250088316D50083124F0884
:1026A0008316D40083124E088316D3007A08DA000A
:1026B0007908D9007808D8007708D7000A12831261
:1026C00065240A166B0884007A08D1007908D000C6
:1026D0007808CF007708CE008A150A16092F6A08F5
:1026E000F2006908F1006808F0006708EF000130A7
:1026F000F300741072088316A3007108A20070081A
:10270000A10083126F088316A0007208D10071081F
:10271000D0007008CF0083126F088316CE00D50159
:10272000D401D301D2010A128312EE260A16031C29
:102730009E2B741480308316A10683128316D10158
:10274000D001CF017E30CE002308D5002208D4006E
:102750002108D3002008D2000A128312EE260A169E
:10276000031C962C83148316D601D501D4017F3027
:10277000D3002308DA002208D9002108D800200855
:10278000D7000A12831265240A1677088316B00050
:102790007808B1007908B2007A08B3003308D10094
:1027A0003208D0003108CF003008CE00D501D40166
:1027B000D3018030D2000A128312A9250A167708A5
:1027C0008316B4007808B5007908B6007A08B70017
:1027D0003708BC003608BB003508BA003408B90019
:1027E0003C08D1003B08D0003A08CF003908CE00A1
:1027F000D501D401D301D2010A128312EE260A16A2
:102800000318042C031D092CF701F801F901FA0142
:102810008A2C83163C08C0003B08BF003A08BE0063
:102820003908BD00BD30C500450884000008C80156
:10283000C7007F304707C9004808CA000318CA0A02
:1028400003104A0CFA00490CF900CB00450884003B
:102850004B0880004008C4003F08C3003E08C20087
:102860003D08C1003C08D1003B08D0003A08CF0029
:102870003908CE004008D5003F08D4003E08D300F8
:102880003D08D2000A128312A9250A168310831666
:102890004008D6003F08D5003E08D4003D08D300CC
:1028A0007A08DA007908D9007808D8007708D700C4
:1028B0000A12831265240A167A088316C000790862
:1028C000BF007808BE007708BD004508840080037B
:1028D0004408D1004308D0004208CF004108CE0090
:1028E0004008D5003F08D4003E08D3003D08D20080
:1028F0000A128312EE260A160319802C83162A2C3C
:1029000083164108F7004208F8004308F90044081C
:10291000FA0083127A088316A3007908A2007808C7
:10292000A1007708A0000230F30783128316230862
:10293000D5002208D4002108D3002008D2002308A3
:10294000D9002208D8002108D7002008D6000A1292
:10295000831276260A167A088316AF007908AE002D
:102960007808AD007708AC003730D500BF30D40010
:102970007D30D300D2002F08D9002E08D8002D08B2
:10298000D7002C08D6000A12831276260A1677087A
:102990008316B0007808B1007908B2007A08B30055
:1029A00083103308D6003208D5003108D40030082F
:1029B000D3003D30DA00AA30D9009330D8008130FE
:1029C000D7000A12831265240A167A088316A70014
:1029D0007908A6007808A5007708A4002708D50084
:1029E0002608D4002508D3002408D2002F08D900D7
:1029F0002E08D8002D08D7002C08D6000A12831202
:102A000076260A1677088316B0007808B100790890
:102A1000B2007A08B30083103308D6003208D5001C
:102A20003108D4003008D300EE30DA005030D9003D
:102A30003330D8008130D7000A12831265240A1679
:102A40007A088316A7007908A6007808A5007708F9
:102A5000A400D501D401D3017F30D2002F08D900C2
:102A60002E08D8002D08D7002C08D6000A12831291
:102A700076260A1677088316B0007808B100790820
:102A8000B2007A08B30083103308D6003208D500AC
:102A90003108D4003008D3000A30DA008D30D90074
:102AA000B130D8008130D7000A12831265240A168B
:102AB0007A088316AB007908AA007808A90077087D
:102AC000A8002B08D5002A08D4002908D30028081C
:102AD000D2002F08D9002E08D8002D08D7002C08C6
:102AE000D6000A12831276260A1677088316B000DB
:102AF0007808B1007908B2007A08B300831033086F
:102B0000D6003208D5003108D4003008D300EE30AA
:102B1000DA005030D9003330D8008130D7000A12A3
:102B2000831265240A167A088316AB007908AA0076
:102B30007808A9007708A8002308D5002208D40047
:102B40002108D3002008D2002708D9002608D80081
:102B50002508D7002408D6000A12831276260A1602
:102B600077088316B0007808B1007908B2007A08B7
:102B7000B300D1003208D0003108CF003008CE00B9
:102B80002B08D5002A08D4002908D3002808D20031
:102B90000A128312A9250A167A088316A700790853
:102BA000A6007808A5007708A400F31C072ED5011D
:102BB000D401D3018030D2002708D9002608D800DC
:102BC0002508D7002408D6000A12831276260A1692
:102BD0008314DB308316D6000F30D5004930D40083
:102BE0007F30D3007A08DA007908D9007808D80055
:102BF0007708D7000A12831265240A167A0883160A
:102C0000A7007908A6007808A5007708A400741C1E
:102C10000B2E8030A506731C2B2E8314DB30D600C0
:102C20000F30D5004930D4007F30D3002708DA00B8
:102C30002608D9002508D8002408D7000A128312D4
:102C400065240A167A088316A7007908A600780872
:102C5000A5007708A4002408F7002508F800260836
:102C6000F9002708FA007A088312EE007908ED00CF
:102C70007808EC007708EB006B08F7006C08F800A8
:102C80006D08F9006E08FA0000345108EA00500897
:102C9000E9004F08E8004E08E7006F237A08D100EA
:102CA0007908D0007808CF007708CE008314DB3095
:102CB0008316D6000F30D5004930D4007F30D300C2
:102CC000831251088316DA00831250088316D90044
:102CD00083124F088316D80083124E088316D7003C
:102CE0000A12831265240A167708E7007808E800BC
:102CF0007908E9007A08EA008316D100831279087E
:102D00008316D000831278088316CF0083127708C9
:102D10008316CE00DB30D5000F30D4004930D3000D
:102D20008030D2000A128312A9250A167708EB0018
:102D30007808EC007908ED007A08EE008316D500DB
:102D4000831279088316D400831278088316D3007F
:102D5000831277088316D200D901D8013430D70006
:102D60008630D6000A12831276260A167708EF00FC
:102D70007808F0007908F1007A08F20083107A08E8
:102D80008316D6007908D5007808D4008312770816
:102D90008316D300DA01D901D8017E30D7000A1298
:102DA000831265240A167A088316D1007908D000A8
:102DB0007808CF007708CE000A1283122F270A1650
:102DC0007808CD008A150A160C2FEB010A12D121C2
:102DD0000A163F08F3000A12C9210A164008F30038
:102DE0000A12C9210A162F30F3000A12C9210A1645
:102DF0004108F3000A12C9210A164208F3000A1218
:102E0000C9210A16303031020139013C031D172F48
:102E1000E30163080A1274200A1600380319162FFA
:102E2000E30AF3000A12C9210A16092F252FE3012C
:102E300063080A127F200A1600380319252FE30AB7
:102E4000F3000A12C9210A16182F5C1C412F300802
:102E5000F3000A12C9210A163108F3000A12C92127
:102E60000A163A30F3000A12C9210A163208F30092
:102E70000A12C9210A163308F3000A12C9210A16D8
:102E80004F2FE30163080A128A200A16003803193B
:102E90004F2FE30AF3000A12C9210A16422F4030CD
:102EA000EB000A12D1210A162E08F3000A12C921DA
:102EB0000A162F08F3000A12C9210A163A30F30045
:102EC0000A12C9210A163008F3000A12C9210A168B
:102ED0003108F3000A12C9210A162030F3000A1241
:102EE000C9210A168A150A16102F6910E801E8018F
:102EF0006808E80A003A03198C2F63306807EA0073
:102F00000A124F230A166A088400780880006808AD
:102F1000033C031C0030782F6918B12F0A124F238D
:102F20000A167808E7006308473C031DA72F6408CA
:102F3000503C031DA72F6508473C031DA72F6608BB
:102F4000473C031DA72F6708413C03196914E80A91
:102F50006408E3006508E4006608E5006708E60029
:102F60008C2F003069180130F8008A150A161A2FC4
:1030000055088316A300831254088316A200831266
:1030100053088316A100831252088316A0000A12D7
:103020008A11831251270A168A157708E700780853
:10303000E8007908E9007A08EA0051088316AB0035
:10304000831250088316AA0083124F088316A90022
:1030500083124E088316A8000A12831255210A16FD
:103060006A088316D500831269088316D400831278
:1030700068088316D300831267088316D2007A0883
:10308000D9007908D8007808D7007708D6000A1246
:103090008A11831276260A168A157708EB007808BB
:1030A000EC007908ED007A08EE0059088316A300B9
:1030B000831258088316A200831257088316A100B2
:1030C000831256088316A0000A128A118312512710
:1030D0000A168A150408EF0083146E088316D600BA
:1030E00083126D088316D50083126C088316D400F2
:1030F00083126B088316D3007A08DA007908D900A6
:103100007808D8007708D7000A128A11831265243C
:103110000A168A156F0884007A08D9007908D80041
:103120007808D7007708D60051088316A3008312C9
:1031300050088316A20083124F088316A100831241
:103140004E088316A0000A128A11831251270A160C
:103150008A1559088316D100831258088316D000A7
:10316000831257088316CF00831256088316CE00A9
:103170007A08D5007908D4007808D3007708D200FF
:103180000A128A118312A9250A168A157A08D10013
:103190007908D0007808CF007708CE00550883164C
:1031A000AB00831254088316AA00831253088316B7
:1031B000A900831252088316A8000A12831255210F
:1031C0000A1651088316D100831250088316D000C6
:1031D00083124F088316CF0083124E088316CE0049
:1031E0007A08D5007908D4007808D3007708D2008F
:1031F0000A128A118312A9250A168A157A08D100A3
:103200007908D0007808CF007708CE005108EA008E
:103210005008E9004F08E8004E08E7008A116F23C4
:103220008A157708E7007808E8007908E9007A0845
:10323000EA008316D100831269088316D000831236
:1032400068088316CF00831267088316CE00DB3030
:10325000D5000F30D4004930D3008030D2000A129C
:103260008A118312A9250A168A157708EB007808B7
:10327000EC007908ED007A08EE008316D500831281
:103280006D088316D40083126C088316D300831252
:103290006B088316D200D901D8013430D7008630AC
:1032A000D6000A128A11831276260A168A157A081F
:1032B000D1007908D0007808CF007708CE00DC1C58
:1032C00063298030CF0683108316D601D5013430B0
:1032D000D4008630D300831251088316DA0083129B
:1032E00050088316D90083124F088316D800831222
:1032F0004E088316D7000A128A11831265240A1613
:103300008A157708E7007808E8007908E9007A0864
:10331000EA0083106A088316D600831269088316B0
:10332000D500831268088316D400831267088316B9
:10333000D300DA01D901D8017E30D7000A128A11F0
:10334000831265240A168A157A088316D100790833
:10335000D0007808CF007708CE000A128A118312B5
:103360002F270A168A157908CC007808CB008A1511
:103370000A160E2F3E08453C031DEB29303039025A
:10338000EA006430F0006A08F1000A128A11202471
:103390000A168A157808EB0030303A02EC000A3041
:1033A000F0006C08F1000A128A1120240A168A150E
:1033B00078086B07ED0030303B026D07EF00F1003D
:1033C0001430F2000A128A117A270A168A15780830
:1033D0004A3EE400172A30303902EA006430F00037
:1033E0006A08F1000A128A1120240A168A15780840
:1033F000EB0030303A02EC000A30F0006C08F100CB
:103400000A128A1120240A168A1578086B07ED0023
:1034100030303B026D07EF00F1001430F2000A1269
:103420008A117A270A168A157808493CE400303058
:103430003402EA000A30F0006A08F1000A128A1128
:1034400020240A168A157808EB00303035026B0705
:10345000ED00F1000A30F2000A128A117A270A16EA
:103460008A1578084A3EE5003E08453C031D672A58
:1034700030303902EA006430F0006A08F1000A12C4
:103480008A1120240A168A157808EB0030303A0297
:10349000EC000A30F0006C08F1000A128A112024B6
:1034A0000A168A1578086B07ED0030303B026D076D
:1034B000EF00F1001430F2000A128A117A270A167E
:1034C0008A150310F70C7708303EE600952A303055
:1034D0003902EA006430F0006A08F1000A128A1129
:1034E00020240A168A157808EB0030303A02EC00E6
:1034F0000A30F0006C08F1000A128A1120240A1622
:103500008A1578086B07ED0030303B026D07EF003D
:10351000F1001430F2000A128A117A270A168A156D
:103520000310F70C7708393CE6003508E7003E0841
:10353000453C031DDC2A30303B020139003A031DB3
:10354000BE2A30303C02EA000A30F0006A08F1007E
:103550000A128A1120240A168A157808EB003030E6
:103560003D026B07ED00F1000530F2000A128A11EE
:103570007A270A168A157808E300DB2A30303C02E5
:10358000EA000A30F0006A08F1000A128A112024C9
:103590000A168A157808EB0030303D026B073C3E76
:1035A000ED00F1000530F2000A128A117A270A169E
:1035B0008A157808E3001D2B30303B020139013CAD
:1035C000031D002B30303C02EA000A30F0006A088C
:1035D000F1000A128A1120240A168A157808EB00D5
:1035E00030303D026B07ED00F1000530F2000A12A9
:1035F0008A117A270A168A1578080B3CE3001D2BDE
:1036000030303C02EA000A30F0006A08F1000A1289
:103610008A1120240A168A157808EB0030303D0202
:103620006B07ED00F1000530F2000A128A117A27CB
:103630000A168A157808173CE30041306307E80052
:1036400030303602EA000A30F0006A08F1000A124F
:103650008A1120240A168A157808EB0030303702C8
:103660006B07ED00F1000530F2000A128A117A278B
:103670000A168A157808E9000310690D413EE90031
:1036800030303602EA000A30F0006A08F1000A120F
:103690008A1120240A168A157808EB003030370288
:1036A0006B07ED00F1000530F2000A128A117A274B
:1036B0000A168A157708E3006308023C031CE90A2E
:1036C0006308023C031D682B3808053C031CE90A0B
:1036D0006408B4006508B5006608B6006708B7005E
:1036E0006808BC006908BD008A150A16122FE3019C
:1036F0000A128A114F230A168A156308043C031C18
:10370000882B0A128A119C230A168A15E30A7D2B3C
:103710000A128A114F230A168A1530307802C70020
:103720000A128A114F230A168A150A128A114F2388
:103730000A168A157808C8000A128A114F230A1639
:103740008A157808C900C70803192F2C0A128A1194
:103750004F230A168A157808C3000A128A114F23CC
:103760000A168A157808C5000A128A114F230A160C
:103770008A157808C60046082E3C031DC32B450851
:10378000C6003030C5004508303C031DD12B46082B
:10379000393C031DD02B3030C6003130C500D12B51
:1037A000C60A30304502E4000A30F0006408F10037
:1037B0000A128A1120240A168A157808E50030308A
:1037C00046026507CA000A128A119C230A168A1546
:1037D0000A128A114F230A168A157808C3000A12A2
:1037E0008A114F230A168A157808C4000A128A1112
:1037F0004F230A168A157808C5000A128A114F232A
:103800000A168A157808C60043082E3C031D0E2CA4
:103810003030C6002030C500C400C30044082E3C30
:10382000031D182C4308C6002030C500C400C30087
:1038300045082E3C031D232C4408C6004308C50040
:103840002030C400C30046082E3C031D2F2C450821
:10385000C6004408C5004308C4002030C3008A15D0
:103860000A16422F20306C1E3030ED006B08F70036
:10387000EB1F412CF709F70A7708EB002D30ED001C
:10388000EC176B08F1006430F2000A128A117A27F3
:103890000A168A157708EB0030307807EE006B08BF
:1038A000F1000A30F2000A128A117A270A168A15E4
:1038B00030307707F00030307807EF006D08F70000
:1038C000EC1D642CEC1F6C116C1A712CEC1F8C2CF1
:1038D0006C198C2C7708EE00EC188C2C7708EF0014
:1038E0008C2C30306E02031D8C2C7708EE002030BB
:1038F000ED00EC1D7F2C6C11EC14EC1FEC10303043
:103900006F02031D8C2C7708EF002030EE00EC1DB9
:103910007F2CEC10EC1F6C106C1D952C6D08F300C7
:103920000A128A11C9210A168A15EC1C9E2C6E08EF
:10393000F3000A128A11C9210A168A156C1CA72CD9
:103940006F08F3000A128A11C9210A168A15700835
:10395000F3000A128A11C9210A168A1500340408D4
:10396000F200EC1FBB2CF217721EF20AEB09EC09F5
:10397000EB0A0319EC0A6C0EF038EE00EE07E23E9B
:10398000EF00323EF1006C080F39EF07EF07F10747
:10399000E93EF000F007F0076B0E0F39F007F10772
:1039A000F00DF10DF109F10D6B080F39F107EE0D76
:1039B0000730ED000A30F107F003031CDB2CF007A1
:1039C000EF03031CDF2CEF07EE03031CE32CEE07D1
:1039D000ED03031CE72C6D30840007307205721371
:1039E00084037205031DFB2C721A840A721AFB2CC5
:1039F0002030F700182D8407713004020319721764
:103A00000008F700031D0C2D721B0C2D721A242DBB
:103A1000F2190C2D2030172DF21F142D2D30F70028
:103A200084037213F213182DF21572123030F70757
:103A3000EC010408EB007708F3000A128A11C9218F
:103A40000A168A156B088400840A721FFC2C8A15DA
:103A50000A16F02D4930EB000A128A11D1210A16FC
:103A60008A156A08F63E0318FD2D0A3E002E203006
:103A7000F3000A128A11C9210A168A153408F300C4
:103A80000A128A11C9210A168A153508F3000A128A
:103A90008A11C9210A168A153608F3000A128A11FA
:103AA000C9210A168A153708F3000A128A11C9219A
:103AB0000A168A153C08F3000A128A11C9210A164F
:103AC0008A153D08F3000A128A11C9210A168A15BF
:103AD000FD2D5C1CA32DC7080319A32DEB016B085A
:103AE0000A128A1194200A168A1500380319802DAB
:103AF000EB0AF3000A128A11C9210A168A156F2DE2
:103B00004308F3000A128A11C9210A168A154408CB
:103B1000F3000A128A11C9210A168A154508F30012
:103B20000A128A11C9210A168A154608F3000A12D8
:103B30008A11C9210A168A156D30F3000A128A11FA
:103B4000C9210A168A15FD2D5C1CC92DC708031949
:103B5000C92D4808F3000A128A11C9210A168A15CC
:103B60004908F3000A128A11C9210A168A15EB01C5
:103B70006B080A128A119B200A168A15003803194D
:103B8000C92DEB0AF3000A128A11C9210A168A15F7
:103B9000B82DFD2D5C1CE62DC7080319E62DEB01A1
:103BA0006B080A128A11A5200A168A150038031913
:103BB000E12DEB0AF3000A128A11C9210A168A15AF
:103BC000D02D4A08EB001130EC003224FD2D5C1C96
:103BD000FC2D033084004C08EC004B08EB00AF2CAC
:103BE0002F30F3000A128A11C9210A168A154D08CE
:103BF000EB001330EC003224FD2D8A150A16A02F9D
:103C00000A108A140A158207372D372D692D692D60
:103C1000A42DA42DE72DE72DCA2D372D84011F30AB
:103C2000830583161F149F141F159F1107309C00D6
:103C30001C0883120D130D30831699002230980052
:103C4000903083129800AC01AD01C701CB01CC01CB
:103C5000CD01DC10FF30DD00E00162140A128A1190
:103C6000DB290A168A152D082C020319A12FE00161
:103C7000621CB32E0A128A11AC210A168A15E301BE
:103C800063080A128A11AF200A168A150038031930
:103C9000512EE30AF3000A128A11C9210A168A1565
:103CA000402E0A128A115F230A168A15F808031992
:103CB0005B2E00305C2E0130F8007818612E621007
:103CC000622E6214621C892E4030EB000A128A11A7
:103CD000D1210A168A15E30163080A128A11BD2050
:103CE0000A168A15003803197D2EE30AF3000A121A
:103CF0008A11C9210A168A156C2E0430E300FA30A5
:103D0000E4000A128A1122210A168A15E30B7F2E7B
:103D1000B22E4030EB000A128A11D1210A168A1500
:103D2000E30163080A128A11CB200A168A150038AB
:103D30000319A22EE30AF3000A128A11C9210A16F6
:103D40008A15912E0430E300FA30E4000A128A1139
:103D500022210A168A15E30BA42E0A128A11AC211D
:103D60000A168A15A02F0A128A115F230A168A15CD
:103D7000F808031DDE2EEB010A128A11D1210A1662
:103D80008A15E30163080A128A11D9200A168A15D6
:103D900000380319D32EE30AF3000A128A11C9214D
:103DA0000A168A15C22E0430E300FA30E4000A1223
:103DB0008A1122210A168A15E30BD52E0A128A11BE
:103DC000A82B0A168A1530303002E400F0000A30C1
:103DD000F1000A128A1120240A168A1530303102A5
:103DE0007807E1005A08610203190E2F6108DA0012
:103DF0000A1200280A160A12302B0A160A12F62C8A
:103E00000A168A1100288A150A126F2F0A168A11BB
:103E10007C298A158A11452E8A1500288A11E52EDB
:103E20008A15BA295B0832020319442F5C1C442FFF
:103E30008A11752F8A15F808031D412FEB010A120C
:103E40008A11D1210A168A15E30163080A128A1120
:103E5000E6200A168A1500380319362FE30AF30004
:103E60000A128A11C9210A168A15252F0430E30087
:103E7000FA30E4000A128A1122210A168A15E30B8D
:103E8000382F772B3208DB004730EB000A128A11FB
:103E9000D1210A168A15C7080319642F5C1C642FE8
:103EA0004A08013C031C642F2130F3000A128A11D6
:103EB000C9210A168A158316061183120615831660
:103EC0008611831286117F2F5C1D6E2F3F30F30009
:103ED0000A128A11C9210A168A15752F2030F3009B
:103EE0000A128A11C9210A168A158316061183122D
:103EF000061183168611831286150430DC063030D5
:103F00003202E400F0000A30F1000A128A11202483
:103F10000A168A157808E500303033027807F70072
:103F20000310F70C7708E800F1000A30F2000A12DB
:103F30008A117A270A168A157708E900EA002A2DDD
:103F4000D42F6008313C0318BD2F0A128A11AC210E
:103F50000A168A15E30163080A128A11F3200A1669
:103F60008A1500380319BC2FE30AF3000A128A11DC
:103F7000C9210A168A15AB2FBE2FE00A83168612B6
:103F8000831286163230E4000A128A1122210A16A0
:103F90008A1583168612831286123230E4000A12C2
:0C3FA0008A1122210A168A15332E6300B4
:02400E00723FFF
:00000001FF
